:0200000480007A
:100000006F008004732F2034930F80006308FF0378
:10001000930F90006304FF03930FB0006300FF038E
:10002000130F000063040F0067000F00732F2034CC
:1000300063540F006F00400093E19153171F0000BD
:1000400023223FFC6FF09FFF93000000130100008C
:10005000930100001302000093020000130300004C
:100060009303000013040000930400001305000034
:10007000930500001306000093060000130700001C
:100080009307000013080000930800001309000004
:1000900093090000130A0000930A0000130B0000EC
:1000A000930B0000130C0000930C0000130D0000D4
:1000B000930D0000130E0000930E0000130F0000BC
:1000C000930F0000732540F16310050097020000B4
:1000D000938202017390523073500018970200000F
:1000E00093824202739052309B021000939252030B
:1000F0009382F2FF7390023B9302F0017390023AF5
:100100007350403097020000938242017390523046
:10011000735020307350303093010000970200007C
:10012000938282EE73905230130510001315F5017F
:10013000635C05000F00F00F930110009308D005D9
:10014000130500007300000093020000638A0200A0
:1001500073905210B7B200009B82921073902230BD
:100160007350003097020000938242017390123462
:10017000732540F17300203097200000938080E8C1
:1001800003E70000B703FF009B83F30F93012000F8
:10019000631E772A972000009380C0E603E74000A3
:1001A000B70301009B8313F093930301938303F040
:1001B00093013000631C772897200000938080E42F
:1001C00003E78000B713F00F9B8303FF9301400008
:1001D000631E7726972000009380C0E203E7C000EB
:1001E000B7030F009B83F30F9393C3009383F30034
:1001F00093015000631C772497200000938040E116
:1002000003E740FFB703FF009B83F30F93016000F8
:10021000631E772297200000938080DF03E780FF32
:10022000B70301009B8313F093930301938303F0BF
:1002300093017000631C772097200000938040DDBD
:1002400003E7C0FFB713F00F9B8303FF9301800008
:10025000631E771E97200000938080DB03E7000079
:10026000B7030F009B83F30F9393C3009383F300B3
:1002700093019000631C771C97200000938080D826
:10028000938000FE83E20002B703FF009B83F30F1D
:100290009301A000639C721A97200000938080D67F
:1002A0009380D0FF83E27000B70301009B8313F0BB
:1002B00093930301938303F09301B0006398721842
:1002C0009301C00013020000972000009380C0D368
:1002D00003E7400013030700B713F00F9B8303FFEE
:1002E000631673161302120093022000E31E52FCE1
:1002F0009301D0001302000097200000938000D1EA
:1003000003E740001300000013030700B7030F00CA
:100310009B83F30F9393C3009383F30063187312CB
:100320001302120093022000E31852FC9301E00034
:1003300013020000972000009380C0CC03E7400028
:10034000130000001300000013030700B7030100AF
:100350009B8313F093930301938303F06318730E4D
:100360001302120093022000E31652FC9301F000E6
:100370001302000097200000938000C903E74000AB
:10038000B713F00F9B8303FF6312770C1302120065
:1003900093022000E31052FE9301000113020000BB
:1003A00097200000938080C61300000003E7400000
:1003B000B7030F009B83F30F9393C3009383F30062
:1003C000631677081302120093022000E31A52FC0E
:1003D000930110011302000097200000938080C257
:1003E000130000001300000003E74000B703010002
:1003F0009B8313F093930301938303F063187704B3
:100400001302120093022000E31852FC972200000E
:10041000938242BF03E102001301200093032000F6
:10042000930120016314710297220000938282BD20
:1004300003E10200130000001301200093032000D9
:100440009301300163147100631030020F00F00F4C
:10045000638001009391110093E111009308D0058E
:1004600013850100730000000F00F00F93011000CE
:100470009308D0051305000073000000731000C03E
:10048000000000000000000000000000000000006C
:10049000000000000000000000000000000000005C
:1004A000000000000000000000000000000000004C
:0C04B00000000000000000000000000040
:1010000000000000000000000000000000000000E0
:1010100000000000000000000000000000000000D0
:1010200000000000000000000000000000000000C0
:1010300000000000000000000000000000000000B0
:081040000000000000000000A8
:10200000FF00FF0000FF00FFF00FF00F0FF00FF0D8
:040000058000000077
:00000001FF
